:104F5C0000000501013C0200000400FA0301FA05FF
:104F6C0000020A0A5A0B000F0C00FA0D00030E0087
:104F7C00030F0132100096120132130AFA140102C7
:104F8C0015010217010A18010A1905321A010A1B28
:104F9C00010A1C053223011E2400642A00FA2B008E
:104FAC00FA2C50782D003C2E00462F001E30006449
:104FBC003250783300003432FA35016436016437EC
:104FCC000050380A643C00643E003C3F000140FF46
:104FDC00FF411450420A5A430AC84405324500782E
:104FEC004600FA47013A4802024C00FA4EFFFF50C5
:104FFC000505510596521432530B28540A96560245
:10500C0002570546580002590A465A32FA5B010A01
:10501C005C14325E000A5F00FE61FFFF64031C66D5
:10502C0000016701036A0A3C6B00006C3296780140
:10503C0032790132FAFAFA0065006F0079008300C8
:10504C008D009700A100AC00B600C000CA00D400CF
:10505C00DE00E800F2005B0063006A0072007A0078
:10506C008200890091009900A100A800B000B8004E
:10507C00BF00C700CF00D600DF00E600EE00F60050
:10508C00400046004C00520059005F0065006B0068
:10509C00710077007D00830089008F0095009C00D3
:1050AC00A200A800AE00B400BA00C000C600CC003C
:0B50BC00D200D900DF00E500EB00F19E
:10009E00AE33AF3474068E048F05FF1200858C3597
:1000AE008D36AE33AF3474068E048F05FF12534A6D
:1000BE008C338D34E534453360137406C39534FFA9
:1000CE00E49533FE8E338F347835125396E550A86F
:1000DE0035B80015D395364010E550C39536FFE47C
:1000EE009535FE8E358F368010E550243CC39536FF
:1000FE00FFE49535FE8E358F36AE35AF36743B6FD9
:10010E004E6006743C6F4E701AAE35AF36743B6F50
:10011E004E7005755001800375500275363A75356F
:10012E000080037550002290009AE0B40104C20BC7
:10013E008002D20B90009BE0B40104C20C8002D26C
:10014E000C9000D8E075F0DCA4FFAEF0740A8E04BB
:10015E008F05FF1200859007C0ECF0A3EDF0A2080A
:10016E00401674038C068D0712532F7401125321FF
:10017E009007BEEEF0A3EFF07E017F00900096E0B8
:10018E0012532F9000D9E08E048F05FF1200857454
:10019E000AFF1200858D399000E2E075F0DCA4FFB5
:1001AE00AEF0740A8E048F05FF1200859007C4EC22
:1001BE00F0A3EDF09000E4E060139000E4E0F5F0C1
:1001CE00741684FF7E00EF9007CCF0800674649066
:1001DE0007CCF09000DEE0B4020674009000C0F090
:1001EE009000DEE0B4020674009000ECF09000C0C7
:1001FE00E0B4020674019000C0F09000ECE0B4018F
:10020E000674009000C0F09000C3E0B40B0874E3D5
:10021E00900085F080499000C3E0B419129000D987
:10022E00E090502E125312E493900085F08030909F
:10023E0000C3E0B41E129000D9E090504C1253123D
:10024E00E493900085F080179000C3E0B4281090DE
:10025E0000D9E0905076125312E493900085F090FE
:10026E0000F6E0B4011790002C740FF0A374FFF0A9
:10027E0090002EE4F0A3F074029000F6F09000F6D9
:10028E00E0B4034190002EE0FEA3E0FF90002CE0CE
:10029E00FCA3E0FD12538E741012532F74081253E8
:1002AE0021EF900082F0EF700674FF900082F074E0
:1002BE00009000F6F090002DE0900083F090002C5E
:1002CE00E0900084F0900087E0900044F0900044AD
:1002DE00E0240C900045F0900044E0241890004675
:1002EE00F0900044E02424900047F0900044E02475
:1002FE0030900048F0900045E0D3943C400B9000C5
:10030E0045E0C3943C900045F0900046E0D3943C09
:10031E00400B900046E0C3943C900046F09000479E
:10032E00E0D3943C400B900047E0C3943C900047D0
:10033E00F0900048E0D3943C400B900048E0C3940A
:10034E003C900048F090004EE4F0900044E0643B96
:10035E006007900044E0B43C20900044E0B43B06BB
:10036E00740290004EF0900044E0B43C0690004EB3
:10037E007401F09000447401F090004FE4F090008E
:10038E0045E0643B6007900045E0B43C209000459A
:10039E00E0B43B06740290004FF0900045E0B43C90
:1003AE000690004F7401F09000457401F0900050DB
:1003BE00E4F0900046E0643B6007900046E0B43CF9
:1003CE0020900046E0B43B067402900050F090007E
:1003DE0046E0B43C069000507401F0900046740163
:1003EE00F0900051E4F0900047E0643B600790000D
:1003FE0047E0B43C20900047E0B43B067402900006
:10040E0051F0900047E0B43C069000517401F0901A
:10041E0000477401F0900052E4F0900048E0643B15
:10042E006007900048E0B43C20900048E0B43B06E2
:10043E007402900052F0900048E0B43C06900052D6
:10044E007401F09000487401F0900087E0FE900077
:10045E00EAE02E900054F0900054E0D3943C400B10
:10046E00900054E0C3943C900054F0900054E0B4DB
:10047E001E06741F900054F0900054E0B43C069099
:10048E0000547401F0900054E0641D600790005415
:10049E00E0B43206900054E014F0900054E0D3948F
:1004AE001E400D900054E0C3941E900055F0800A3B
:1004BE00900054E0241E900055F09000CDE0900086
:1004CE0049F0900049E0640B6017900049E0641712
:1004DE00600F900049E064236007900049E0B42F5C
:1004EE0006900049E014F0900049E0640C6017900B
:1004FE000049E06418600F900049E06424600790A2
:10050E000049E0B43006900049E004F0900049E064
:10051E00240C90004AF0900049E0241890004BF013
:10052E00900049E0242490004CF0900049E02430E3
:10053E0090004DF090004AE0D3943C400B90004A5E
:10054E00E0C3943C90004AF090004BE0D3943C40C2
:10055E000B90004BE0C3943C90004BF090004CE0AD
:10056E00D3943C400B90004CE0C3943C90004CF074
:10057E0090004DE0D3943C400B90004DE0C3943C72
:10058E0090004DF022C293C294C291C292C287C211
:10059E0090E5B554EFF5B5E5B554DFF5B5C296C2A5
:1005AE0095C2A0C297C2A2C2A1E5B5547FF5B5E52A
:1005BE00B554BFF5B5E5B554FBF5B5C20D75374667
:1005CE009000D0E0700575490280037549039000D4
:1005DE001474FFF0A374DCF09000B1E090001AF8F0
:1005EE00E4F0E8A3F0C213C215C217C219C21B74FD
:1005FE00C8900030F074C8900034F074C890003881
:10060E00F074C890003CF074C8900040F07526005D
:10061E00752500C208756C00E54BB40903754B00D7
:10062E00753C00900022E4F0A3F0754C1E75280076
:10063E00752700C210C211C2129007C0E0FEA3E0DF
:10064E00FF740312532F74011253219007BEEEF064
:10065E00A3EFF0C203900018E4F0A3F0C22122052C
:10066E003D2285A74F75A710A2D8B34002C293A210
:10067E00D9B34002C294A2DAB34002C291A2DBB354
:10068E004002C292A2DCB34002C28775D840854FA9
:10069E00A722900047E4936406600280FE74C8901F
:1006AE0007C6F8E4F0E8A3F075B50075840175A7E8
:1006BE000075FF8075EF06900053E4F075C9107554
:1006CE00A70F75A1C775A70075D90075CE0C75A7B4
:1006DE000F75F1FE75F2FF75F30775F47875A4BA10
:1006EE0075A5FF75A60775AE0075AFFF75D481753C
:1006FE00D5FF75D6FF75D7FF75A70075A20175A139
:10070E004775F80975D80075D90475A71075D80006
:10071E0075D90475DA0975DB0975DC0975DD09759E
:10072E00DE0975D84075A70075E60075E71075BC33
:10073E000175BE0475BD6C75BE0775BDA075BE088E
:10074E0075BD0175BC0075BB1875BC2075BA0875F2
:10075E00E88075D11375B50075A70F75E10575E2C3
:10076E000075C740C293C294C291C292C287C29012
:10077E00E5B554EFF5B5E5B554DFF5B5C296C295BE
:10078E00C2A0C297C2A2C2A1E5B5547FF5B5E5B528
:10079E0054BFF5B5E5B554FBF5B575970075978063
:1007AE00740A1200757597C0E5975420700280F890
:1007BE00758F0275A700D2AF75980075A90C75A735
:1007CE000F75AB4375ADFB75AC1E75A71075C918CB
:1007DE0075CA0075CB0075C80475A70075891275AA
:1007EE008E04758C00758A00C2A9D28C758D007529
:1007FE008B00D2ABD28E75D944753200753100752F
:10080E002E00752D00754600754700C29974C8F507
:10081E00097508001233B275B50074639007C6F8F7
:10082E00E4F0E8A3F012363E7464F5097508001280
:10083E0033B2C220900070E0B40108A2B54002D2DB
:10084E0020802E900070E0B4021175A70F75F30F83
:10085E0075A700A2A34002D2208016900070E0B4CB
:10086E00030F75A70F75F31775A700A2A44002D248
:10087E0020A220B3500302096D74089007C6F8E455
:10088E00F0E8A3F012350D7464F509750800123303
:10089E00B274099007C6F8E4F0E8A3F012350D74AF
:1008AE0064F5097508001233B2740A9007C6F8E4AD
:1008BE00F0E8A3F012350D7464F5097508001233D3
:1008CE00B2740B9007C6F8E4F0E8A3F012350D747D
:1008DE0064F5097508001233B2740C9007C6F8E47B
:1008EE00F0E8A3F012350D7464F5097508001233A3
:1008FE00B2740D9007C6F8E4F0E8A3F012350D744B
:10090E0064F5097508001233B2740E9007C6F8E448
:10091E00F0E8A3F012350D7464F509750800123372
:10092E00B274029000CFF0900070E0900093F090BF
:10093E000070E0B40108740090009BF0801C9000E1
:10094E0070E0B4020874009000DEF0800D9000702C
:10095E00E0B4030674009000EBF0D21E020A4D9034
:10096E0007C6E4F0A304F012350D7464F50975089A
:10097E00001233B274029007C6F8E4F0E8A3F01246
:10098E00350D7464F5097508001233B274039007BF
:10099E00C6F8E4F0E8A3F012350D7464F509750895
:1009AE00001233B274049007C6F8E4F0E8A3F01214
:1009BE00350D7464F5097508001233B2740590078D
:1009CE00C6F8E4F0E8A3F012350D7464F509750865
:1009DE00001233B274069007C6F8E4F0E8A3F012E2
:1009EE00350D7464F5097508001233B2740790075B
:1009FE00C6F8E4F0E8A3F012350D7464F509750835
:100A0E00001233B274019000CFF0900070E09000AD
:100A1E0093F0900070E0B40108740090009BF08099
:100A2E001C900070E0B4020874009000DEF0800D9F
:100A3E00900070E0B4030674009000EBF0C21E123A
:100A4E0037B29000D9E07006740A9000D9F0900089
:100A5E0085E0700674E3900085F0120135E5B5442B
:100A6E0001F5B5740690005FF07401900060F074AB
:100A7E0003900062F07404900063F0741D900064A3
:100A8E00F07405900065F07403900066F0740090A9
:100A9E00006BF0740090006CF0740190006DF074B7
:100AAE000090006EF074FF90006FF0743690015D50
:100ABE00F0743090015EF0742D90015FF0743290FE
:100ACE000160F07420900161F07435900162F07451
:100ADE0043900163F07479900164F0746C90016539
:100AEE00F07420900166F07420900167F0742090ED
:100AFE000168F07420900169F0742090016AF0741E
:100B0E002090016BF09000F5E0900082F09000AC28
:100B1E00E0900083F09000ADE0900084F0C213C22C
:100B2E0015C217C219C21B74C8900030F074C89059
:100B3E000034F074C8900038F074C890003CF07423
:100B4E00C8900040F0C210C211C212A2B6B39209F0
:100B5E00A2B3B3920A752600752500753746754CFB
:100B6E001E90007EE4F075271975286490001474A9
:100B7E00FFF0A374DCF0C20D754B00C208752A009D
:100B8E00752900900018E4F0A3F0743A900786F0EF
:100B9E0074FD900787F0756D0090007FE4F0752C62
:100BAE0000752B0090001CE4F0A3F09000B1E090D3
:100BBE00001AF8E4F0E8A3F0900092E075F032A489
:100BCE00FFAEF090002AEEF0A3EFF09007C0E0FE2B
:100BDE00A3E0FF740312532F74011253219007BE2A
:100BEE00EEF0A3EFF0754A0174FA90005BF0C221AB
:100BFE00756C00753C00C20EC20FC222C203754D49
:100C0E0000C204D205C206D207D21F74FE9000564F
:100C1E00F074FE900057F0753800754400753A0078
:100C2E00753E32753F00754000743C900059F0746B
:100C3E003C90005AF07541007542007543009000DB
:100C4E0022E4F0A3F0754500D2B2D2A4D2B0D2B154
:100C5E00D2A3D2A7D2A6D2A5D2B7900092E0D394B7
:100C6E00FA400674FA900092F07E017F00900084A4
:100C7E00E012532F900083E02FFF50010E90002CB6
:100C8E00EEF0A3EFF0EFD394FFEE940F4007900039
:100C9E002CE4F0A3F0900082E0700674FF900082C6
:100CAE00F09000CFE0D39402400674019000CFF094
:100CBE009000D0E0700575490280037549039000DD
:100CCE00D1E0D39401400674009000D1F09000D78B
:100CDE00E0C3940A5006740A9000D7F09000E1E049
:100CEE00700674019000E1F09000E1E0B4FF06742C
:100CFE00FE9000E1F09000E8E0D394FE400674FE12
:100D0E009000E8F074019000EEF074019000EFF0A6
:100D1E0074009000F1F074009000F6F0D29CD2ECCA
:100D2E0075CF01A298B35003021124C298E547640F
:100D3E00046006E59964FF6002801EE54760087452
:100D4E00E6254790005BF0754700E546600874F0B5
:100D5E00254690005BF0754600E5476003020E09DC
:100D6E00754700E599B4FF03754601E599B4FE0396
:100D7E00754602E599B4FD03754603E599B4FC0387
:100D8E00754604E599B4FA03754605E599B4FB0377
:100D9E00754701E599B4F903754704E599D394E5D0
:100DAE004007E599C394F04002801685994875472F
:100DBE00027E017F00E548C394E612532F8E2F8FDB
:100DCE0030753200753100E599D394C74007E59927
:100DDE00C394E64002801F85994875470374E5C3A6
:100DEE009548F530752F00AE2FAF309050C71200DA
:100DFE00647831125374D299021124E547B401027A
:100E0E008003020EE7E53245317003120593AE31D1
:100E1E00AF32900086125356E599F0783112539600
:100E2E00AE31AF32EFB40106EEB407028003020E0C
:100E3E00E7900786E0B43C028003020ED1C29C12FA
:100E4E000135900082E09000F5F0900083E0900074
:100E5E00ACF0900084E09000ADF0A21E40327550D0
:100E6E0001E550D394075026E5509007C6F8E4F0FC
:100E7E00E8A3F074AA900053F01233DE7464F509FF
:100E8E007508001233B27850740126F650D38030B4
:100E9E00755008E550D3940E5026E5509007C6F8CD
:100EAE00E4F0E8A3F074AA900053F01233DE7464F9
:100EBE00F5097508001233B27850740126F650D336
:100ECE001237B274C89007C6F8E4F0E8A3F0D29CCB
:100EDE007547007546007599FBE547B4020280031D
:100EEE00020F7BE5324531700685992E752D00AEC9
:100EFE0031AF3274016F4E701BAC2DAD2EAA2FABDD
:100F0E0030ED2BFBEC3AFA8A068B079000861253D3
:100F1E0056E599F07831125396AE31AF3274026FB6
:100F2E004E704AAC2DAD2E740D6D4C7027746390BF
:100F3E0007C6F8E4F0E8A3F074AB900053F090000D
:100F4E0093E0900070F012371774C89007C6F8E45B
:100F5E00F0E8A3F0AE2DAF2E74566F4E700312054F
:100F6E0093120135854899754700754600E547B4DB
:100F7E00033FAE31AF32900086125356E599F078AA
:100F8E0031125396AE31AF32AC2FAD308F028E038D
:100F9E008C068D07905103120064E493F97401934B
:100FAE00FEEAD39EEB994009854899754700754630
:100FBE0000E547B404028003021124E53245317086
:100FCE0003120593AE31AF32900086125356E59957
:100FDE00F07831125396AE31AF32EFB40006EEB464
:100FEE0001028003021124900069E075F002A4FD55
:100FFE00ACF08D50ED90008612536BEDFAE0FBEAEB
:10100E0090008912536BEBFAE0FBEA2BFA90006921
:10101E00E0B5020280030211150DED900086125309
:10102E006BE550FDE0FAED90008A12536BEAFDE09D
:10103E00FAEDC39AFD900069E0B505028003021136
:10104E0015E55090008812536BE550FDE0FAED90D7
:10105E00008B12536BEAFDE0FAED2AFD900069E079
:10106E00B505028003021115E55090008C12536BEA
:10107E00FDE0FAED900069E0F4042A900070F0E5CE
:10108E005090008D12536BFDE0FAED900069E0F484
:10109E00042A900071F0E55090008E12536BFDE023
:1010AE00FAED900069E0F4042A900072F0E5509099
:1010BE00008F12536BFDE0FAED900069E0F4042A04
:1010CE009007C6F8E4F0E8A3F074AB900053F0126A
:1010DE0037177464F5097508001233B29007C612FB
:1010EE00533D1237177464F5097508001233B29028
:1010FE0007C612533D1237177599F97464F50975C1
:10110E0008001233B280FE7599FF7464F5097508F4
:10111E00001233B280FEE5466006A299B3B34003D7
:10112E00021285C299E546B4011FAE31AF3290006E
:10113E005F125356E0F5997831125396AE31AF32B5
:10114E0074116F4E7003754600E546B40203854A6E
:10115E0099E546B4031DAE31AF3290008612535658
:10116E00E0F599EFB40107EEB40703754600783148
:10117E00125396E546B404028003021264E532452A
:10118E00317003852699AE31AF3274016F4E700304
:10119E00853899AE31AF3274026F4E7003853A992D
:1011AE00AE31AF3274036F4E7003853E99AE31AFE0
:1011BE003274046F4E7003854099AE31AF327405B0
:1011CE006F4E7003854199AE31AF3274066F4E701B
:1011DE0003854299AE31AF3274076F4E700385436B
:1011EE0099AE31AF3274086F4E7006900023E0F561
:1011FE0099AE31AF3274096F4E700690005BE0F518
:10120E0099AE31AF32740A6F4E7003854499AE3188
:10121E00AF32740B6F4E7003853F99AE31AF32749F
:10122E000C6F4E7003854599AE31AF32740D6F4E13
:10123E00700590005BE4F0AE31AF32740D6F4E70FE
:10124E00037599FC7831125396AE31AF32740E6F2E
:10125E004E7003754600E546B4051CAE31AF3290B4
:10126E004F5C125356E493F59974E66F4E70037506
:10127E0046007831125396E54764016005E547B4A0
:10128E000403020D2EC28E7E107F00E53D12532FF9
:10129E00E58D75F010A4FDACF0EF2DFDEE3CFCE5F8
:1012AE008B75F01084FF7E00ED2FFFEC3EFE8E2737
:1012BE008F28D28E9000B3E0605690002412533DDA
:1012CE00900024E0FCA3E0FD900026E0FAA3E0FBF2
:1012DE00EDB5033CECB50238B21DA208B34013A223
:1012EE001DB34008E5B54404F5B58006E5B554FBDD
:1012FE00F5B5900026E0FEA3E0FF900028E0FCA3E9
:10130E00E0FDEF2DFDEE3CFC900026ECF0A3EDF0A1
:10131E009000ECE060030213D59000C0E0600990ED
:10132E0000C0E0C394034002807A124CB2A208B30C
:10133E00500990007EE0C39446400280069000AAB9
:10134E00E0F56BE56B75F005A4FFAEF09007C8EE07
:10135E00F0A3EFF0900097E0C3953A4007E538C34D
:10136E00953950079007C8E4F0A3F0AE58AF5990E6
:10137E0007C8E0FCA3E0FDEFD39DEE9C4004C2A1A4
:10138E00800B90007EE0C394645002D2A19000C006
:10139E00E0B402099000DEE0C3940240028005A290
:1013AE00A1B392A29000C0E0B4031C124DAEAE5891
:1013BE00AF599007C8E0FCA3E0FDEFD39DEE9C4033
:1013CE0004D2A18002C2A1A2B6300901B350030219
:1013DE00192EA2B6300901B3500302192EA2B6304F
:1013EE000B01B35003021848754A009000B3E07029
:1013FE0013A20BB34008E5B554FBF5B58006E5B571
:10140E004404F5B50537A20DB3B35013AE27AF287C
:10141E00900014E0FCA3E0FDEDC39FEC9E400302A0
:10142E00150BE549B40330E537B43B05754901802A
:10143E001FA221B3401AE537C3943B500690005BC0
:10144E007401F0E537D3943B4006740290005BF0D4
:10145E00753701D2218044E549B4020675490175FC
:10146E00373BE537B43B05753701802F90005BE0C5
:10147E00701AE537C3943B500690005B7401F0E59B
:10148E0037D3943B4006740290005BF09000D0E09E
:10149E00B402051205938003753701AE29AF2AAC4D
:1014AE0027AD28EF2DFDEE3CFC74028C068D071245
:1014BE0053218E298F2A9000B3E0603F900024E0E4
:1014CE00FCA3E0FD9000B3E0FF12008574018C06D2
:1014DE008D07125321900028EEF0A3EFF090002814
:1014EE00E0F8A3E0900026C8F0A3C8F0900024E432
:1014FE00F0A3F0C21DE5B554FBF5B5802BAE29AFB8
:10150E002AAC27AD28EF2DFDEE3CFC74018C068D28
:10151E00071253218E298F2AAC27AD28EDD394B80C
:10152E00EC940B4003120593E537B43B1074039013
:10153E00005BF09000D0E0B40203120593AE2BAF27
:10154E002CAC27AD28EF2DFDEE3CFC8C2B8D2CAE5C
:10155E0027AF28EFD39DEE9C401190001CE0FAA31C
:10156E00E0FBEBC394E8EA94034002800690001C73
:10157E0012533D900018E0FEA3E0FFAC27AD28EF1C
:10158E002DFDEE3CFC900018ECF0A3EDF09000D099
:10159E00E0B40218AE27AF28740512532F7401124F
:1015AE005321900014EEF0A3EFF08011AE27AF2878
:1015BE00740212532F900014EEF0A3EFF0C28E754A
:1015CE008D00758B00753D00752801752700D28E34
:1015DE00E537240E75F00F84AFF07E00EF4E707578
:1015EE00900018E0F8A3E0900016C8F0A3C8F090A1
:1015FE000016E0FEA3E0FFEF4E600B7C817D5A12D9
:10160E0052318E258F26900018E4F0A3F0AE25AF50
:10161E00267428BE00039F5010E53C2FFF50010E8C
:10162E0074011253218E258F2685263C9000D7E01B
:10163E00A825B8000DD395264008E526900058F051
:10164E0080099000D7E014900058F0E549600675C7
:10165E002600752500E537640B6005E537B42909CA
:10166E009000C0E060031249F4900054E0653760CA
:10167E0007900055E0B53703754B00A20E500302DC
:10168E00176990008CE0B4015AE54075F00584FFAF
:10169E007E00900586125356E0F534753300AE3356
:1016AE00AF3490008AE012532F74648E048F05FFBE
:1016BE0012008574C18C068D0712532F8E358F360E
:1016CE0090001AE0FEA3E0FFAC33AD3412000374B9
:1016DE00648E048F05FF12008590001AECF0A3EDC6
:1016EE00F0800F90008AE075F0C1A4FFAEF08E3549
:1016FE008F36E53AC394CC506075A71085F95085A6
:10170E00FA517E017F00E55112532FE5502FFF5005
:10171E00010E8E338F34AC35AD36EF2DFDEE3CFC25
:10172E008C358D36D293D294D291D292D287E53621
:10173E00F5FBE535F5FCE536F5E9E535F5EAE53693
:10174E00F5EBE535F5ECE536F5EDE535F5EEE5369B
:10175E00F5FDE535F5FE75A700D20EE549B4010697
:10176E00E53764116002800F754C0190005E7401C4
:10177E00F0E5B54401F5B5E5496003021843900064
:10178E00D3E0600D9000DAE0A825B800069526405B
:10179E0002804A9000D3E0B4022F900044E06537F7
:1017AE00601F900045E065376017900046E0653792
:1017BE00600F900047E065376007900048E0B5374E
:1017CE0003754C03754500800CC2007545009000F2
:1017DE0022E4F0A3F0740990005BF080589000446E
:1017EE00E0B5370B754C0190005E7401F0804690A9
:1017FE000045E0B5370B754C01740290005EF08029
:10180E0034900046E0B5370B754C01740390005EC2
:10181E00F08022900047E0B5370B754C01740490B0
:10182E00005EF08010900048E0B53709754C0174E9
:10183E000590005EF0A20BB39209A20BB330B60175
:10184E00B3500302192E754A019000B3E07013A233
:10185E000BB34008E5B54404F5B58006E5B554FB79
:10186E00F5B5A20B9209E537D3944A4012D20DE595
:10187E0037D394854009740390005BF0753746901A
:10188E0000DBE0B40107E543C39414400280031269
:10189E000593744690007EF0A204300501B35017F4
:1018AE00A204B34008E5B54408F5B58006E5B55485
:1018BE00F7F5B5A2049205A206300701B35017A2A0
:1018CE0006B34008E5B54402F5B58006E5B554FD0E
:1018DE00F5B5A2069207E543C394415009740E90E4
:1018EE00005BF0120593900065E0FE900061E0C38E
:1018FE009E4009900061E0D39406400974FB90006D
:10190E005BF012059390006AE0601590006AE0FEAD
:10191E00900064E06E600974FE90005BF012059317
:10192E00A210B3B35008900049E0653760028060A2
:10193E00A202B35006A200B3B34002804D9000EC59
:10194E00E0600BA203B34004D2A18002C2A175A72E
:10195E001085F95085FA517E017F00E55112532F03
:10196E00E5502FFF50010E8E338F34900020E0FC97
:10197E00A3E0FDEF2DFDEE3CFC8C358D36E536F506
:10198E00FBE535F5FC75A700D293C210D211D21229
:10199E00A211B3B3500890004AE065376002806030
:1019AE00A202B35006A200B3B34002804D9000ECE9
:1019BE00E0600BA203B34004D2A18002C2A175A7BE
:1019CE001085F95085FA517E017F00E55112532F93
:1019DE00E5502FFF50010E8E338F34900020E0FC27
:1019EE00A3E0FDEF2DFDEE3CFC8C358D36E536F596
:1019FE00E9E535F5EA75A700D294D210C211D212DC
:101A0E00A212B3B3500890004BE0653760028060BD
:101A1E00A202B35006A200B3B34002804D9000EC78
:101A2E00E0600BA203B34004D2A18002C2A175A74D
:101A3E001085F95085FA517E017F00E55112532F22
:101A4E00E5502FFF50010E8E338F34900020E0FCB6
:101A5E00A3E0FDEF2DFDEE3CFC8C358D36E536F525
:101A6E00EBE535F5EC75A700D291D210D211C2126A
:101A7E00A210B3B3500890004CE06537600280604E
:101A8E00A202B35006A200B3B34002804D9000EC08
:101A9E00E0600BA203B34004D2A18002C2A175A7DD
:101AAE001085F95085FA517E017F00E55112532FB2
:101ABE00E5502FFF50010E8E338F34900020E0FC46
:101ACE00A3E0FDEF2DFDEE3CFC8C358D36E536F5B5
:101ADE00EDE535F5EE75A700D292C210D211D212F5
:101AEE00A211B3B3500890004DE0653760028060DC
:101AFE00A202B35006A200B3B34002804D9000EC98
:101B0E00E0600BA203B34004D2A18002C2A175A76C
:101B1E001085F95085FA517E017F00E55112532F41
:101B2E00E5502FFF50010E8E338F34900020E0FCD5
:101B3E00A3E0FDEF2DFDEE3CFC8C358D36E536F544
:101B4E00FDE535F5FE75A700D287D210C211D2126F
:101B5E00E54CB40818124323A210B35005A211B3DA
:101B6E0040028006D210D211D212754C1EE54CB432
:101B7E0007061240DB754C08E54CB4063D90001A82
:101B8E00E0FEA3E0FFEF4E6006A208B3B340028072
:101B9E0023AE52AF5390001AE0FCA3E0FDEF2DFDF3
:101BAE00EE3CFC8C528D53E537D3940A50069000D0
:101BBE001A120039123EAD754C07E54CB4050612EB
:101BCE003D0D754C06E54CB404329000C1E09033E7
:101BDE0094F82828731239A180121239A1800D129F
:0C1BEE003B4F8008123C018003123C01B8
:0F339400021BE3021BE8021BED021BF2021BF7F8
:101BFA009000A3E06005124ADD8002C204754C051C
:101C0A00E54CB403028003021CF49000A6E06005D0
:101C1A00124BCD8002C2069000C1E0D39402403F2D
:101C2A00900095E02403A825B80004952650099051
:101C3A000097E0D3953A50028008D20274089000C7
:101C4A005BF0900095E0A825B80005D39526500BC7
:101C5A00900097E02403C3953A5002C2028039905B
:101C6A000095E02403A825B8000495265007E53816
:101C7A00C3953940028008D202740890005BF09044
:101C8A000095E0A825B80005D395265009E5392422
:101C9A000FC395385002C2029000DBE07007E5439B
:101CAA00C3941440028002D202A2024005754C0479
:101CBA00800A754C1E900022E4F0A3F0A208B340FB
:101CCA0029E54075F00584FF7E009005861253567B
:101CDA00E0C394695005124A29800F9007C0E0F8C2
:101CEA00A3E09007BEC8F0A3C8F0E54CB40A02808E
:101CFA0003021DB6900032E0C394465008C296749F
:101D0A0046900032F090004EE0B4011DE55A2406D8
:101D1A00F55A9007C2E0FEA3E0FF74062FFF5001B8
:101D2A000E9007C2EEF0A3EFF090004EE0B4021D51
:101D3A00E55A240CF55A9007C2E0FEA3E0FF740CA2
:101D4A002FFF50010E9007C2EEF0A3EFF0855A3430
:101D5A00753300900044E0F55012009EE53690007D
:101D6A0032F090000AE533F0A3E534F0E550900034
:101D7A0033F0C2149007C2E0F533A3E0F5349000C3
:101D8A0044E0F55012009EE536900030F0900000D5
:101D9A00E533F0A3E534F0E550900031F0C213E5E5
:101DAA0049B40105754C0B8003754C03900030E073
:101DBA00B537028003021E55A2134072900000E05C
:101DCA00FEA3E0FFEF4E6021AE29AF2A900000E0AB
:101DDA00FCA3E0FD12000374068E048F05FF1200B7
:101DEA0085900000ECF0A3EDF0900031E0601A90CD
:101DFA000000E0FEA3E0FFAC29AD2AEF2DFDEE3C8A
:101E0A00FC900000ECF0A3EDF0900031E0D39401D7
:101E1A00401A900000E0FEA3E0FFAC29AD2AEF2DA6
:101E2A00FDEE3CFC900000ECF0A3EDF0D213AE27DF
:101E3A00AF28900000E0FCA3E0FDEFC39DEE9C40BC
:101E4A000AD296C21374C8900030F0A213B3B350EA
:101E5A0007900030E0B53702800AD29674C8900025
:101E6A0030F0C213900032E0B537028003021F0D32
:101E7A00A214407290000AE0FEA3E0FFEF4E602138
:101E8A00AE29AF2A90000AE0FCA3E0FD1200037419
:101E9A00068E048F05FF12008590000AECF0A3ED70
:101EAA00F0900033E0601A90000AE0FEA3E0FFAC75
:101EBA0029AD2AEF2DFDEE3CFC90000AECF0A3EDD3
:101ECA00F0900033E0D39401401A90000AE0FEA398
:101EDA00E0FFAC29AD2AEF2DFDEE3CFC90000AECA8
:101EEA00F0A3EDF0D214AE27AF2890000AE0FCA3CD
:101EFA00E0FDEFC39DEE9C400AC296744690003204
:101F0A00F0C214A214B3B35007900032E0B53702FE
:101F1A00800AC2967446900032F0C214E54CB40BA3
:101F2A00028003021FE8900036E0C394465008C2BC
:101F3A00957446900036F090004FE0B4011DE55AC2
:101F4A002406F55A9007C2E0FEA3E0FF74062FFFAD
:101F5A0050010E9007C2EEF0A3EFF090004FE0B4EC
:101F6A00021DE55A240CF55A9007C2E0FEA3E0FFD1
:101F7A00740C2FFF50010E9007C2EEF0A3EFF0850C
:101F8A005A34753300900045E0F55012009EE5364C
:101F9A00900036F090000CE533F0A3E534F0E550FC
:101FAA00900037F0C2169007C2E0F533A3E0F5348B
:101FBA00900045E0F55012009EE536900034F0900E
:101FCA000002E533F0A3E534F0E550900035F0C2A5
:101FDA0015E549B40105754C0C8003754C03900056
:101FEA0034E0B537028003022087A21540729000C0
:101FFA0002E0FEA3E0FFEF4E6021AE29AF2A900077
:10200A0002E0FCA3E0FD12000374068E048F05FFB4
:10201A00120085900002ECF0A3EDF0900035E0602C
:10202A001A900002E0FEA3E0FFAC29AD2AEF2DFDD5
:10203A00EE3CFC900002ECF0A3EDF0900035E0D30A
:10204A009401401A900002E0FEA3E0FFAC29AD2AF9
:10205A00EF2DFDEE3CFC900002ECF0A3EDF0D21562
:10206A00AE27AF28900002E0FCA3E0FDEFC39DEE8F
:10207A009C400AD295C21574C8900034F0A215B3D8
:10208A00B35007900034E0B53702800AD29574C87D
:10209A00900034F0C215900036E0B5370280030292
:1020AA00213FA216407290000CE0FEA3E0FFEF4E23
:1020BA006021AE29AF2A90000CE0FCA3E0FD1200DB
:1020CA000374068E048F05FF12008590000CECF055
:1020DA00A3EDF0900037E0601A90000CE0FEA3E058
:1020EA00FFAC29AD2AEF2DFDEE3CFC90000CECF084
:1020FA00A3EDF0900037E0D39401401A90000CE071
:10210A00FEA3E0FFAC29AD2AEF2DFDEE3CFC9000CA
:10211A000CECF0A3EDF0D216AE27AF2890000CE03D
:10212A00FCA3E0FDEFC39DEE9C400AC29574469065
:10213A000036F0C216A216B3B35007900036E0B5C7
:10214A003702800AC2957446900036F0C216E54CF2
:10215A00B40C02800302221A90003AE0C39446505B
:10216A0008C2A0744690003AF0900050E0B4011DF5
:10217A00E55A2406F55A9007C2E0FEA3E0FF74066A
:10218A002FFF50010E9007C2EEF0A3EFF09000501F
:10219A00E0B4021DE55A240CF55A9007C2E0FEA3EA
:1021AA00E0FF740C2FFF50010E9007C2EEF0A3EF70
:1021BA00F0855A34753300900046E0F55012009EBF
:1021CA00E53690003AF090000EE533F0A3E534F0DE
:1021DA00E55090003BF0C2189007C2E0F533A3E047
:1021EA00F534900046E0F55012009EE5369000382E
:1021FA00F0900004E533F0A3E534F0E5509000399F
:10220A00F0C217E549B40105754C0D8003754C03FE
:10221A00900038E0B5370280030222B9A217407253
:10222A00900004E0FEA3E0FFEF4E6021AE29AF2A42
:10223A00900004E0FCA3E0FD12000374068E048FF4
:10224A0005FF120085900004ECF0A3EDF090003930
:10225A00E0601A900004E0FEA3E0FFAC29AD2AEF8B
:10226A002DFDEE3CFC900004ECF0A3EDF09000395B
:10227A00E0D39401401A900004E0FEA3E0FFAC29E9
:10228A00AD2AEF2DFDEE3CFC900004ECF0A3EDF03E
:10229A00D217AE27AF28900004E0FCA3E0FDEFC3FD
:1022AA009DEE9C400AD2A0C21774C8900038F0A2D2
:1022BA0017B3B35007900038E0B53702800AD2A0AE
:1022CA0074C8900038F0C21790003AE0B53702801F
:1022DA0003022371A218407290000EE0FEA3E0FFF1
:1022EA00EF4E6021AE29AF2A90000EE0FCA3E0FD7C
:1022FA0012000374068E048F05FF12008590000EEB
:10230A00ECF0A3EDF090003BE0601A90000EE0FEC6
:10231A00A3E0FFAC29AD2AEF2DFDEE3CFC90000EA8
:10232A00ECF0A3EDF090003BE0D39401401A90004A
:10233A000EE0FEA3E0FFAC29AD2AEF2DFDEE3CFC3A
:10234A0090000EECF0A3EDF0D218AE27AF28900063
:10235A000EE0FCA3E0FDEFC39DEE9C400AC2A07410
:10236A004690003AF0C218A218B3B3500790003A48
:10237A00E0B53702800AC2A0744690003AF0C2184B
:10238A00E54CB40D02800302244C90003EE0C39455
:10239A00465008C297744690003EF0900051E0B44F
:1023AA00011DE55A2406F55A9007C2E0FEA3E0FF94
:1023BA0074062FFF50010E9007C2EEF0A3EFF090C3
:1023CA000051E0B4021DE55A240CF55A9007C2E008
:1023DA00FEA3E0FF740C2FFF50010E9007C2EEF02F
:1023EA00A3EFF0855A34753300900047E0F5501298
:1023FA00009EE53690003EF0900010E533F0A3E52C
:10240A0034F0E55090003FF0C21A9007C2E0F5336D
:10241A00A3E0F534900047E0F55012009EE53690AF
:10242A00003CF0900006E533F0A3E534F0E5509067
:10243A00003DF0C219E549B40105754C0E800375DB
:10244A004C0390003CE0B5370280030224EBA2194A
:10245A004072900006E0FEA3E0FFEF4E6021AE2935
:10246A00AF2A900006E0FCA3E0FD12000374068E7A
:10247A00048F05FF120085900006ECF0A3EDF090A2
:10248A00003DE0601A900006E0FEA3E0FFAC29AD33
:10249A002AEF2DFDEE3CFC900006ECF0A3EDF09047
:1024AA00003DE0D39401401A900006E0FEA3E0FF4D
:1024BA00AC29AD2AEF2DFDEE3CFC900006ECF0A312
:1024CA00EDF0D219AE27AF28900006E0FCA3E0FD9C
:1024DA00EFC39DEE9C400AD297C21974C890003C83
:1024EA00F0A219B3B3500790003CE0B53702800A56
:1024FA00D29774C890003CF0C21990003EE0B537FC
:10250A000280030225A3A21A4072900010E0FEA3E3
:10251A00E0FFEF4E6021AE29AF2A900010E0FCA345
:10252A00E0FD12000374068E048F05FF12008590E9
:10253A000010ECF0A3EDF090003FE0601A9000105C
:10254A00E0FEA3E0FFAC29AD2AEF2DFDEE3CFC90A6
:10255A000010ECF0A3EDF090003FE0D39401401A94
:10256A00900010E0FEA3E0FFAC29AD2AEF2DFDEEAE
:10257A003CFC900010ECF0A3EDF0D21AAE27AF2885
:10258A00900010E0FCA3E0FDEFC39DEE9C400AC260
:10259A0097744690003EF0C21AA21AB3B35007903D
:1025AA00003EE0B53702800AC297744690003EF0BA
:1025BA00C21AE54CB40E02800302269A900042E049
:1025CA00C394465008C2A27446900042F09000524A
:1025DA00E0B4011DE55A2406F55A9007C2E0FEA3AD
:1025EA00E0FF74062FFF50010E9007C2EEF0A3EF32
:1025FA00F0900052E0B4021DE55A240CF55A9007F7
:10260A00C2E0FEA3E0FF740C2FFF50010E9007C238
:10261A00EEF0A3EFF0855A34753300900048E0F5E8
:10262A005012009EE536900042F0900012E533F019
:10263A00A3E534F0E550900043F0C21C9007C2E0D5
:10264A00F533A3E0F534900048E0F55012009EE51A
:10265A0036900040F0900008E533F0A3E534F0E549
:10266A0050900041F0C21BE549B40121754900743C
:10267A00C8900030F074C8900034F074C8900038E4
:10268A00F074C890003CF074C8900040F0754C0398
:10269A00900040E0B537028003022739A21B40723E
:1026AA00900008E0FEA3E0FFEF4E6021AE29AF2ABA
:1026BA00900008E0FCA3E0FD12000374068E048F6C
:1026CA0005FF120085900008ECF0A3EDF0900041A0
:1026DA00E0601A900008E0FEA3E0FFAC29AD2AEF03
:1026EA002DFDEE3CFC900008ECF0A3EDF0900041CB
:1026FA00E0D39401401A900008E0FEA3E0FFAC2961
:10270A00AD2AEF2DFDEE3CFC900008ECF0A3EDF0B5
:10271A00D21BAE27AF28900008E0FCA3E0FDEFC370
:10272A009DEE9C400AD2A2C21B74C8900040F0A23F
:10273A001BB3B35007900040E0B53702800AD2A21B
:10274A0074C8900040F0C21B900042E0B537028086
:10275A00030227F1A21C4072900012E0FEA3E0FFE0
:10276A00EF4E6021AE29AF2A900012E0FCA3E0FDF3
:10277A0012000374068E048F05FF12008590001262
:10278A00ECF0A3EDF0900043E0601A900012E0FE36
:10279A00A3E0FFAC29AD2AEF2DFDEE3CFC90001220
:1027AA00ECF0A3EDF0900043E0D39401401A9000BE
:1027BA0012E0FEA3E0FFAC29AD2AEF2DFDEE3CFCB2
:1027CA00900012ECF0A3EDF0D21CAE27AF289000D7
:1027DA0012E0FCA3E0FDEFC39DEE9C400AC2A27486
:1027EA0046900042F0C21CA21CB3B35007900042AC
:1027FA00E0B53702800AC2A27446900042F0C21CB9
:10280A00E54CB4020280030228A812478C1248A39E
:10281A009007BEE0FEA3E0FF740A12532F90001641
:10282A00E0FCA3E0FD74098F02FF1200858D078C7E
:10283A00038E048A058B061252319007C2EEF0A36A
:10284A00EFF074F0BE00039F500B74F09007C2F8CB
:10285A00E4F0E8A3F09007C2E0FEA3E0FFE55A2FF8
:10286A00FF50010E9007C2EEF0A3EFF090005EE079
:10287A00B40103754C0A90005EE0B40203754C0B78
:10288A0090005EE0B40303754C0C90005EE0B40463
:10289A0003754C0D90005EE0B40503754C0EE54CD3
:1028AA00B401259000F3E09033A3F8282873124569
:1028BA002A801212452A800D1245B48008124660F9
:0528CA008003124660CE
:0F33A3000228B80228BD0228C20228C70228CC7F
:1028CF00754C029000DEE0B4020280030229EA9008
:1028DF000081E0D3953F5064900081E0F404253FE0
:1028EF00FE9000E1E08E00F5F0E884FF7E008F504F
:1028FF00EFC39410500CEF8550F0A4FDACF08D5049
:10290F0080037550FF900081E0D39550400B9000ED
:10291F0081E0C39550F54D8003754D009000FCE0AC
:10292F00D3954D40069000FCE0F54D9000FDE0C3BF
:10293F00954D50069000FDE0F54D8071900081E0BF
:10294F00C3953FFE9000E1E08E00F5F0E884FF7E36
:10295F00008F50EFC39410500CEF8550F0A4FDACD6
:10296F00F08D5080037550FF855034753300900003
:10297F0081E02534FFAE3350010E8E338F3474FF58
:10298F00BE0009D39F400585344D8003754DFF90E0
:10299F0000FCE0D3954D40069000FCE0F54D900013
:1029AF00FDE0C3954D50069000FDE0F54DA208B334
:1029BF00B350099000E9E0D3954E5002800A740796
:1029CF0090005BF0C2A1801375A710E5CDC3954DA4
:1029DF004004C2A18002D2A175A700E54BC39409A0
:1029EF004003023125A2EDB35003023125C2EDE5BC
:1029FF004B6003022B9990008FE07003022B88909D
:102A0F0000C5E0B401028003022AE8900054E0B54B
:102A1F0037028003022AE57E017F00E5BE12532FA5
:102A2F00E5BD2FFF50010E8E338F3490008FE0B431
:102A3F000118741012532F900085E08E048F05FF3C
:102A4F00120085ED900056F0802CAE33AF34741029
:102A5F0012532F900085E08E048F05FF1200859092
:102A6F000056E02DFD50010C74018C068D0712539A
:102A7F0021EF900056F0E54460089000EBE064020F
:102A8F00600280219000EDE0B4011A900056E075CD
:102A9F00F0E7A4FFAEF0E5448E048F05FF1200852A
:102AAF00ED900056F0900056E0FE900057E0D39E58
:102ABF004004D21F8002B21F900056E0900057F0E2
:102ACF009000C1E064016006A21FB3B3400280060C
:102ADF00900056E0F538022B86D21F7E017F00E56D
:102AEF00BE12532FE5BD2FFF50010E8E338F349042
:102AFF00008FE0B40118741012532F900085E08EF0
:102B0F00048F05FF120085ED900056F0802CAE3338
:102B1F00AF34741012532F900085E08E048F05FF91
:102B2F00120085900056E02DFD50010C74018C06AB
:102B3F008D07125321EF900056F0E5446008900086
:102B4F00EBE06402600280219000EDE0B4011A9086
:102B5F000056E075F0E7A4FFAEF0E5448E048F0554
:102B6F00FF120085ED900056F09000C1E064016007
:102B7F0006900056E0F538800375380090008BE022
:102B8F007005754B01800375BB18E54BB4010280CE
:102B9F0003022D3B90008BE07003022D2A7E017FF4
:102BAF0000E5BE12532FE5BD2FFF50010E8E338F60
:102BBF00349000D1E0B4010F7E0F7FFFAC33AD3402
:102BCF0012538E8E338F349000F6E0B40245AE333D
:102BDF00AF3490002CE0FCA3E0FDEDD39FEC9E40C2
:102BEF000A90002CE533F0A3E534F0AE33AF349008
:102BFF00002EE0FCA3E0FDEFD39DEE9C400A900079
:102C0F002EE533F0A3E534F0AE33AF347404125332
:102C1F00218F3A9000F6E0704CAE33AF3490002C19
:102C2F00E0FCA3E0FDEFD39DEE9C400912538E8E86
:102C3F00338F348006753400753300AE33AF347480
:102C4F001012532F900082E08E048F05FF12008523
:102C5F008C338D347400D39D74019C400585343AB8
:102C6F008003753AFF9000C1E0B401028003022D8A
:102C7F0028A208B3B3500E900095E0A825B8000520
:102C8F00D395265003022D1D900096E075F019A4E0
:102C9F00FFAEF09000D9E08E048F05FF12008590F3
:102CAF0000D2E0853AF0A4FFAEF074648D028C037D
:102CBF008E048F05FF120085EA2DFDEB3CFC8C3353
:102CCF008D34E544600F9000EBE0B402089000ED06
:102CDF00E0640160028017AE33AF3474E712532FF4
:102CEF00E5448E048F05FF1200858C338D349000E0
:102CFF0056E0A833B8000AD39534400585343880A0
:102D0F000BA21FB34006900056E0F538800BA21FB0
:102D1F00B34006900056E0F5388003753A009000F6
:102D2F008EE07005754B02800375BB19E54BB4023D
:102D3F00028003022DF690008EE07003022DE5E570
:102D4F0037D3941E4003022DE390002AE0FEA3E048
:102D5F00FFE53E12538690002AEEF0A3EFF07E01BE
:102D6F007F00E5BE12532FE5BD2FFF50010E8E33AE
:102D7F008F349000FBE07013740A12532F74518E2E
:102D8F00048F05FF1200858D3E8019AE33AF34746A
:102D9F000A12532F8F048E057E017F95CDCCCD1255
:102DAF0052318F3EE53ED394644003753E649000EC
:102DBF002AE0FEA3E0FFE53E2FFF50010E90002A10
:102DCF00EEF0A3EFF0900092E0048E048F05FF1257
:102DDF0000858D3E8003753E329000DEE0700575F4
:102DEF004B03800375BB13E54BB4035E9000DEE02D
:102DFF0060477E017F00E5BE12532FE5BD2FFF50C8
:102E0F00010E8E338F3474041253218F3F9000E0E4
:102E1F00E0853FF0A4FDACF07464FF1200858D3F98
:102E2F009000DFE0853FF0A4FFAEF074FF8E048FBB
:102E3F0005FF1200858D4E8003753F0090008CE0DA
:102E4F007005754B04800375BB17E54BB404028006
:102E5F0003022EF790008CE0B4017C7E017F00E529
:102E6F00BE12532FE5BD2FFF50010E7404125321D4
:102E7F008E338F34900059E06012900059E0149017
:102E8F00513F93A833B80006953440028006900056
:102E9F0059E014F0900059E0C39477501390005903
:102EAF00E00490513F93A833B80005D395345002F6
:102EBF008006900059E004F0900059E0FE9000B2B7
:102ECF00E08E0088F0A4FFAEF074648E048F05FFCF
:102EDF001200858D40800375400090008DE07005D5
:102EEF00754B05800375BB16E54BB40502800302D5
:102EFF002F8A90008DE0B4017C7E017F00E5BE1229
:102F0F00532FE5BD2FFF50010E74041253218E3342
:102F1F008F3490005AE0601290005AE0149051B82C
:102F2F0093A833B8000695344002800690005AE00B
:102F3F0014F090005AE0C39477501390005AE004B5
:102F4F009051B893A833B80005D39534500280063A
:102F5F0090005AE004F090005AE0FE9000B8E08E26
:102F6F000088F0A4FFAEF074648E048F05FF12008A
:102F7F00858D41800375410075BB1FE54BB406334A
:102F8F007E017F00E5BE12532FE5BD2FFF50010ECE
:102F9F008E338F34740912532F74E68E048F05FF0E
:102FAF001200858D43900094E07005754B078003E8
:102FBF0075BB15E54BB4070280030230CC9000942B
:102FCF00E070030230BB7E017F00E5BE12532FE598
:102FDF00BD2FFF50010E8E338F3474041253218F87
:102FEF0042900094E0B401159000E8E08542F0A40F
:102FFF00FFAEF07407125321EF9007CBF0900094BF
:10300F00E0B402159000E8E08542F0A4FFAEF07442
:10301F0007125321EF9007CAF0900094E0B4030217
:10302F0080030230B99000D5E0701CE542C3940ACA
:10303F005002D201E542D394644002C2019000B421
:10304F00E0900080F080639000B4E070349000E86E
:10305F00E08542F0A4FFAEF074FF8E048F05FF12DF
:10306F000085ED900080F0AE25AF26741EBE0006E1
:10307F00D39F4002D201E53AD394E54002C20180CA
:10308F0029E542C3940A500DAE25AF26741EBE002B
:10309F0004D39F50028002D201E53AD394E5400257
:1030AF00C2019000B4E0900080F080037542009060
:1030BF0000EBE07005754B08800375BB14E54BB44E
:1030CF0008509000EBE060397E017F00E5BE12539F
:1030DF002FE5BD2FFF50010E8E338F34EFD3942188
:1030EF00EE940E40057544FF8015AE33AF34741067
:1030FF0012532F74E38E048F05FF1200858D4480C9
:10310F000375440090008FE0600575BB1A8003754E
:10311F00BB18054BD2ECAE27AF28EFD39428EE9413
:10312F00235003023391C20D7537469000D0E070E3
:10313F00057549028003754903C293C294C291C2B7
:10314F0092C287C290E5B554EFF5B5E5B554DFF5FA
:10315F00B5C296C295C2A0C297C2A2C2A1E5B5548C
:10316F007FF5B5E5B554BFF5B5A220B34008E5B579
:10317F004404F5B58006E5B554FBF5B5A20FB35081
:10318F000EE53AD394334007E53AC394CC4003029B
:10319F00322DE5B54401F5B5744690007EF09000F0
:1031AF008AE075F064A4FFAEF08E358F367402BEE0
:1031BF00000AD39F400675360275350075A7108536
:1031CF00F95085FA517E017F00E55112532FE550DA
:1031DF002FFF50010E8E338F34AC35AD36EF2DFDF2
:1031EF00EE3CFC8C358D36D293D294D291D292D2C2
:1031FF0087E536F5FBE535F5FCE536F5E9E535F51B
:10320F00EAE536F5EBE535F5ECE536F5EDE535F5C3
:10321F00EEE536F5FDE535F5FE75A700D20FE53A7B
:10322F00C3941A5002C20F90001474FFF0A374DC01
:10323F00F09000B1E090001AF8E4F0E8A3F0C213A8
:10324F00C215C21774C8900030F074C8900034F0E3
:10325F0074C8900038F074C890003CF0C210C211CE
:10326F00752600752500753C00C208756C0090002E
:10327F0022E4F0A3F0754C1E9007C0E0FEA3E0FF20
:10328F00740312532F74011253219007BEEEF0A353
:10329F00EFF09000A3E06005124ADD8002C20490B7
:1032AF0000A6E06005124BCD8002C206A2043005D5
:1032BF0001B35017A204B34008E5B54408F5B58033
:1032CF0006E5B554F7F5B5A2049205A2063007013D
:1032DF00B35017A206B34008E5B54402F5B5800612
:1032EF00E5B554FDF5B5A2069207C203752C00751E
:1032FF002B0090001CE4F0A3F0900092E075F032E8
:10330F00A4FFAEF090002AEEF0A3EFF0900018E4C7
:10331F00F0A3F0C22190007FE0C3943C5019758D4B
:10332F0031758B00753D02E54BB4090990007FE0C4
:10333F0004F0754B00803BE54BB40903754B0075EA
:10334F002800752700758D00758B00753D00900066
:10335F007EE0C39464500890007EE004F080067411
:10336F006490007EF090007EE0B46406E5B554FEF4
:10337F00F5B5E543C394415009740E90005BF0120C
:05338F000593020D2E64
:1050C7000000010001400160018001A001C001E072
:1050D70002000300039603B603D603F40400050099
:1050E70005180530054805600578059005A805C031
:1050F700060006140628063C066E068C00FF013FD4
:10510700015F017F019F01BF01DF01FF02FF0395DF
:1051170003B503D503F303FF04FF0517052F054761
:10512700055F0577058F05A705BF05FF061306274A
:10513700063B066F068B06A9DAD8D7D5D4D2D0CFCF
:10514700CDCBC9C7C6C4C2C0BEBCBAB8B5B3B1AF70
:10515700ADABA8A6A4A2A09D9B99969492908D8B87
:1051670089878482807E7C79777573716F6D6B69AF
:10517700676563615F5D5B5957565452504F4D4B9E
:105187004A4847454442413F3E3C3B3A393736352A
:10519700343231302F2E2D2C2B2A2928272625254E
:1051A7002423222121201F1E1E1D1C1C1B1A1A1915
:1051B70019EEECEBEAE9E8E7E5E4E3E1E0DEDDDB65
:1051C700D9D8D6D4D2D0CECCCAC8C6C3C1BFBCBA30
:1051D700B7B5B2B0ADABA8A5A3A09D9B989592908B
:1051E7008D8A8785827F7D7A7775726F6D6A68652C
:1051F70063615E5C5A575553514F4D4B4947454381
:1052070042403E3C3B393836353332312F2E2D2B39
:105217002A292827262524232221201F1E1D1D1C5D
:0A5227001B1A1A191818171616158D
:1033B200750B00750A00AE0AAF0BAC08AD09EDC380
:1033C2009FEC9E401674FF12007575CF01780B7446
:1033D2000126F6500418E436F650DB22900053E042
:1033E200B4AA1C900786E0B43C159007C6E0FEA381
:1033F200E0FFEF4E6009741EBE0004D39F5003022B
:10340200350C75360075350075F8099007C6E0FE73
:10341200A3E0FF74076F4E6006740E6F4E70067461
:103422003A900786F09007C6E0FEA3E0FF7408BE5C
:10343200001ED39F401A7E017F089007C6E0FCA3BE
:10344200E0FD1DBDFF011C1200038E338F34801F6F
:103452009007C6E0FEA3E0FF74081253868F048E25
:10346200057E017F08CDCCCD1200038E338F34AEA2
:1034720035AF36740CD39F74019E5003023507A2F8
:10348200F9B3407EE5364535700375A382AE35AF9C
:103492003674016F4E700375A300AE35AF367402F9
:1034A2006F4E700D9007C7E075F002A4FDACF08D71
:1034B200A3AE35AF3674036F4E700375A300AE35FD
:1034C200AF367403BE00039F5013AC33AD34ED2FFF
:1034D200FFEC3EFE900082125356E0F5A3AE35AFEC
:1034E20036EFB40B09EEB401057414120075AE3553
:1034F200AF36EFB40B07EEB4010375F80D78351251
:103502005396023471900053E4F0227536007535FB
:103512000075F8099007C6E0FEA3E0FF7408BE003C
:103522001ED39F401A7E017F089007C6E0FCA3E0ED
:10353200FD1DBDFF011C1200038E338F34801F90CE
:1035420007C6E0FEA3E0FF74081253868F048E05BF
:103552007E017F08CDCCCD1200038E338F34AE3581
:10356200AF367411D39F74019E500302363DA2F907
:10357200B3500302363AE5364535700375A3D2AE31
:1035820035AF3674016F4E700375A300AE35AF369A
:1035920074026F4E700D9007C7E075F002A4FDAC87
:1035A200F08DA3AE35AF3674036F4E700375A30072
:1035B200AE35AF3674046F4E700375A300AE35AFEF
:1035C2003674056F4E700375A300AE35AF367406C0
:1035D2006F4E700375A300AE35AF3674076F4E7031
:1035E2000375A300AE35AF3674086F4E700375A332
:1035F20000AE35AF367408BE00039F5016AC33AD33
:1036020034ED2FFFEC3EFE90007D125356E5A3F001
:1036120075A300AE35AF36EFB41009EEB4010574F0
:1036220014120075AE35AF36EFB41007EEB40103D5
:1036320075F80D783512539602356022753600758D
:10364200350075F809AE35AF367417BE0004D39F46
:103652005003023716A2F9B35003023713E5364579
:1036620035700375A3D2AE35AF3674016F4E700359
:1036720075A300AE35AF3674026F4E700D9007C75A
:10368200E075F002A4FDACF08DA3AE35AF36740345
:103692006F4E700375A300AE35AF3674046F4E7073
:1036A2000375A300AE35AF3674056F4E700375A374
:1036B20000AE35AF3674066F4E700375A300AE359B
:1036C200AF3674076F4E700375A300AE35AF367414
:1036D200086F4E700375A300AE35AF367408BE0096
:1036E200039F500C900067125356E5A3F075A30098
:1036F200AE35AF3674166F4E70057414120075AE87
:1037020035AF3674166F4E700375F80D7835125357
:103712009602364722900053E0B4AB028003023790
:10372200B175360075350075F809AE35AF367412CD
:10373200BE007CD39F4078A2F9B34070E536453590
:10374200700375A382AE35AF3674016F4E70037588
:10375200A300AE35AF3674026F4E700D9007C7E00E
:1037620075F002A4FDACF08DA3AE35AF3674036FD5
:103772004E700375A300AE35AF367403BE00039FCF
:10378200500990006C125356E0F5A3AE35AF367473
:10379200116F4E70057414120075AE35AF36741188
:1037A2006F4E700375F80D783512539602372C223E
:1037B20090005CE4F074649007C6F8E4F0E8A3F0CB
:1037C20012363E74C89007C6F8E4F0E8A3F0900001
:1037D20073E0B4371A900070E0900067F0900071C7
:1037E200E0900068F0900072E0900069F0804690EE
:1037F200005C7401F074659007C6F8E4F0E8A3F089
:1038020012363E74C89007C6F8E4F0E8A3F09000C0
:1038120073E0B4371A900070E0900067F090007186
:10382200E0900068F0900072E0900069F080067409
:103832000290005CF090005DE4F074669007C6F8B8
:10384200E4F0E8A3F012363E74C89007C6F8E4F03C
:10385200E8A3F0900072E0B43712900070E090009C
:1038620061F0900071E090006AF0807690005D74E3
:1038720001F074679007C6F8E4F0E8A3F012363E50
:1038820074C89007C6F8E4F0E8A3F0900072E0B4C0
:103892003712900070E0900061F0900071E09000AB
:1038A2006AF0803E740290005DF074689007C6F87A
:1038B200E4F0E8A3F012363E74C89007C6F8E4F0CC
:1038C200E8A3F0900072E0B43712900070E090002C
:1038D20061F0900071E090006AF08006740390003D
:1038E2005DF022E55D2534FFAE3350010E90008677
:1038F200125356E0F55EE55D2534FFAE3350010EFE
:103902000FBF00010E900086125356E0F55F8565E9
:1039120061E55EB55F05855E5D8041E55FD3955EDD
:10392200401DE55FC3955E8560F0A4FFAEF0E561E2
:103932008E048F05FF120085ED255EF55D801DE585
:103942005EC3955F8560F0A4FFAEF0E5618E048FE3
:1039520005FF120085EDF404255EF55D22E55FD3D7
:10396200955E401DE55FC3955E8560F0A4FFAEF0F5
:10397200E5618E048F05FF120085ED255EF55D8001
:103982001DE55EC3955F8560F0A4FFAEF0E5618E34
:10399200048F05FF120085EDF404255EF55D22E536
:1039A2003875F00484FF7E008F5DE53875F004847D
:1039B200ADF07C008D60756504753301753400E5EA
:1039C2005DC3943F50051238E580069001C5E0F5CD
:1039D2005D855D53755200900058E075F020A4FF9C
:1039E200AEF09000D7E08E048F05FF1200858D5D4A
:1039F2009000BFE0D395385003023AA79000E3E06D
:103A0200D395384010ED9001C612536BE0F5557511
:103A12005400023AA49000AEE0D395384043E55DED
:103A22009001C612536BE0F55EE55D9001E612531C
:103A32006BE0F55F9000E3E0F4042538F560900058
:103A4200AEE0FE9000E3E0F4042EF561E55EB55FC2
:103A520005855E5D800312395F855D557554008072
:103A620041E55D9001E612536BE0F55EE55D900283
:103A72000612536BE0F55F9000AEE0F4042538F5D2
:103A8200609000BFE0FE9000AEE0F4042EF561E528
:103A92005EB55F05855E5D800312395F855D557594
:103AA2005400023B4E9000E6E0D395385011E55D9C
:103AB20090024612536BE0F555755400023B4E904E
:103AC20000AFE0D395385043E55D90022612536B68
:103AD200E0F55EE55D90024612536BE0F55F900003
:103AE200AFE0F4042538F5609000E6E0FE9000AF08
:103AF200E0F4042EF561E55EB55F05855E5D800349
:103B020012395F855D557554008041E55D9002066E
:103B120012536BE0F55EE55D90022612536BE0F501
:103B22005F9000BFE0F4042538F5609000AFE0FE3E
:103B32009000BFE0F4042EF561E55EB55F05855E99
:103B42005D800312395F855D55755400229000F740
:103B5200E0F562756511753302753400AE25AF2646
:103B6200E56275F00FA4FDACF0EDD39FEC9E402111
:103B7200E5628E048F05FF120085ED75F010A4FF3B
:103B8200AEF0E53875F01184FD7C00ED2FF5638011
:103B92000EE53875F01184FF7E00EF24F0F56385A1
:103BA200635DE53875F01184AFF07E008F601238E6
:103BB200E5855D64AE25AF269000F7E075F00FA4B1
:103BC200FDACF0EDD39FEC9E4028753302753410A6
:103BD20085635D1238E585645E855D5FAE25AF263F
:103BE200E5628E048F05FF12534A8D608562611271
:103BF200395F855D53755200755564755400229086
:103C020000F7E0F562756511753302753400AE2573
:103C1200AF26E56275F00FA4FDACF0EDD39FEC9EEC
:103C22004021E5628E048F05FF120085ED75F010CC
:103C3200A4FFAEF0E53A75F01184FD7C00ED2FF59E
:103C420063800EE53A75F01184FF7E00EF24F0F5F3
:103C52006385635DE53A75F01184AFF07E008F6095
:103C62001238E5855D64AE25AF269000F7E075F069
:103C72000FA4FDACF0EDD39FEC9E40287533027586
:103C8200341085635D1238E585645E855D5FAE251F
:103C9200AF26E5628E048F05FF12534A8D6085625E
:103CA2006112395F855D537552009000C1E0B40422
:103CB20053E53875F00484FF7E008F5DE53875F0BA
:103CC2000484ADF07C008D60756504753301753434
:103CD20000E55DC3943F50051238E580069001C5AA
:103CE200E0F55DAE52AF53E55D12532F74648E045E
:103CF2008F05FF120085AE52AF53EF2DFDEE3CFC57
:103D02008C528D537555647554002290008CE0B42A
:103D12000146E54075F00584FF7E008F5DE5407544
:103D2200F00584ADF07C008D607565057533057511
:103D32003400E55DC3941750051238E580069005FE
:103D42009DE0F55DAE54AF55E55D2FFF50010E7459
:103D5200641253868E548F5590008DE0B40146E56F
:103D62004175F00584FF7E008F5DE54175F00584A5
:103D7200ADF07C008D60756505753305753448E5D9
:103D82005DC3941750051238E580069005E5E0F50D
:103D92005DAE54AF55E55D2FFF50010E74641253B2
:103DA200868E548F5590009CE0B40249E543C3943B
:103DB2004175F00584FF7E008F5DE54375F0058453
:103DC200ADF07C008D60756505753306753400E5D0
:103DD2005DC3941350051238E58006900699E0F50C
:103DE2005DAE54AF55E55D2FFF50010E7464125362
:103DF200868E548F559000DEE0B402028003023EAC
:103E0200ACE53875F01584FF7E008F5DE53875F0FE
:103E12001584ADF07C008D607565157533037534BE
:103E2200F4E55DC3940B50051238E58006900485D5
:103E3200E0F55DE55D75F0FFA4FFAEF09000DFE018
:103E42008E048F05FF120085ED900081F0E53F752D
:103E5200F078A4FFAEF074FF8E048F05FF12008588
:103E62008C338D3474028C068D071253218F5DAC16
:103E720033AD347404FF12534A8D60756504753393
:103E82000675346EE55DC3941D50051238E5800653
:103E9200900711E0F55DAE54AF55E55D2FFF50017F
:103EA2000E74641253868E548F5522900094E0B49F
:103EB20001179007CBE02555FFAE5450010E90003C
:103EC200E8E01253868E548F55900094E0B40316A6
:103ED200A201B3B35010900080E0C39405A825B8A6
:103EE20000069526400280109000B6E02555FFAEF0
:103EF2005450010E8E548F5590008EE0B402028011
:103F0200030240DA900091E0602FE540D3941E4016
:103F12002890001CE0FEA3E0FF9000CCE075F003C7
:103F2200A4FDACF0EFD39DEE9C400E9000F0E0A813
:103F320025B80005D3952650030240DA9000D9E057
:103F42008538F0A4FFAEF0740512532F7407125394
:103F5200218E338F34900098E0A825B8000495266E
:103F62005012900099E075F002A4FDACF0EFC39DF1
:103F7200EE9C40030240DAE53875F00B84FF7E00C8
:103F8200900616125356FEE0FFEE900090E0FEEF10
:103F92008E0088F0A4FFAEF074648E048F05FF12C9
:103FA20000858C338D34900058E075F018A4FFAE74
:103FB200F09000D7E08E048F05FF1200858C068DED
:103FC2000790062E125356AE33AF34E012532F74BD
:103FD200648E048F05FF1200858C338D34E53EA874
:103FE20033B80077D395344072E53EC39534FFE48D
:103FF2009533FE8E338F347428BE00039F500C75A8
:104002003428753300740D90005BF0AE33AF3490FA
:104012000091E012532F74288E048F05FF12008541
:104022008C338D34AE52AF53740A8E048F05FF1257
:1040320000858D068C07AC33AD34CFCECF12000392
:10404200740A8E048F05FF1200858C338D34AE52B4
:10405200AF5312538E8E528F53807DE53EA833B8F4
:10406200000495345072AE33AF34E53E1253868E5F
:10407200338F347428BE00039F500C753428753377
:1040820000740D90005BF0AE33AF34900091E012FB
:10409200532F74288E048F05FF1200858C338D34C4
:1040A200AE52AF53740A8E048F05FF1200858D063F
:1040B2008C07AC33AD34CFCECF120003740A8E041A
:1040C2008F05FF1200858C338D34AE52AF53EF2D26
:1040D200FDEE3CFC8C528D5322AE52AF53AC54AD2C
:1040E2005512000374648E048F05FF1200858C52F2
:1040F2008D53900089E08C068D0712532F74648EC5
:10410200048F05FF1200858C528D53A2084017AE12
:1041120025AF267405BE00039F5002D208E53AD3AC
:1041220094CC4002D2029000EBE0B402089000ED81
:10413200E0640160028017AE52AF53E54412532F80
:1041420074E78E048F05FF1200858C528D53900008
:10415200ABE05402601B9000A2E0A825B80012D385
:104162009526400DA208B3B35007E53AC3949A408E
:10417200028028AE5BAF5C9000A0E075F002A4FD67
:10418200ACF0EF2DFDEE3CFC74022DFD50010CE570
:104192003ABC0007D39D4003756901853A5C755BA3
:1041A20000E56970030242319000FEE0C395694068
:1041B20070E54075F00584FF7E0090058612535627
:1041C200E0F534753300AE33AF349000B0E01253F3
:1041D2002F74648E048F05FF1200858C358D369006
:1041E20000FEE004C395698C068D0712532F9000E0
:1041F200FEE08E048F05FF1200858C358D3690000F
:10420200A1E08C068D0712532F740A8E048F05FFCE
:10421200120085AE52AF53EF2DFDEE3CFC8C528D59
:104222005305699000FEE0C39569500375690090DB
:1042320000ABE05401601B90009FE0A825B800127B
:10424200D39526400DA208B3B35007E538C394CCEA
:104252004002802590009DE075F003A4FFAEF0E5DA
:10426200662FFF50010E74032FFF50010EE538BE7A
:104272000007D39F4003756A01853866E56A7003BB
:1042820002430C9000FFE0C3956A4070E54075F070
:104292000584FF7E00900586125356E0F53475338F
:1042A20000AE33AF349000B0E012532F74648E042A
:1042B2008F05FF1200858C358D369000FFE004C318
:1042C200956A8C068D0712532F9000FFE08E048FA3
:1042D20005FF1200858C358D3690009EE08C068D90
:1042E2000712532F740A8E048F05FF120085AE52F7
:1042F200AF53EF2DFDEE3CFC8C528D53056A9000BE
:10430200FFE0C3956A5003756A009000B0E0A852BE
:10431200B80004955350099000B0E0F5537552006F
:10432200229000ECE0B40102800302442EA208B302
:10433200500302442C9000B7E0B40168AE52AF5370
:10434200AC25AD26120003743C8E048F05FF1200CB
:10435200859000C7E0BC00109D400D9000C9E0A808
:1043620052B8000495535002D203AE52AF53AC255B
:10437200AD26120003743C8E048F05FF1200859057
:1043820000C7E0C3940ABC0015D39D40119000C938
:10439200E0C39405A852B80005D395535002800299
:1043A200C2038068AE52AF53AC25AD26120003742F
:1043B200788E048F05FF1200859000C7E0BC0010C4
:1043C2009D400D9000C9E0A852B8000495535004D6
:1043D200D2038038AE52AF53AC25AD26120003741F
:1043E200788E048F05FF1200859000C7E0C3940AFF
:1043F200BC0015D39D40119000C9E0C39405A8529A
:10440200B80005D3955350028002C203A203B34001
:1044120019AE52AF539000C8E012532F74648E0449
:104422008F05FF1200858C528D538002C2039000CB
:10443200ECE0B40258E53875F00884FF7E008F5D29
:10444200E53875F00884ADF07C008D6075650875FF
:1044520033017534E0E55DC3943F50051238E580C1
:1044620006900285E0F55DE55D75F05EA4FFAEF0B5
:10447200740A8E048F05FF1200858C568D577402C4
:10448200BC000AD39D4006755702755600A200B3C0
:104492004006A202B3B35009900022E4F0A3F080D8
:1044A20024AE52AF537400D39F74019E400C90000F
:1044B20022E552F0A3E553F0800B74FF900022F83E
:1044C200E4F0E8A3F09000CEE0D394024006A20804
:1044D200B3B34002800DAE52AF53740212532F8E0B
:1044E200528F539000B7E0B4010DAE52AF53740235
:1044F20012532F8E528F53AE52AF53745E12532FFC
:10450200740A8E048F05FF1200858C528D5374023B
:10451200BC000AD39D4006755302755200900020DC
:10452200E552F0A3E553F022900058E09003861282
:10453200536BE0F567756864900058E0FE9000C226
:10454200E0D39E4037E53875F00884FF7E008F5D2A
:10455200E53875F00884ADF07C008D6075650875EE
:104562003303753496E55DC3941F50051238E58018
:104572000690043BE0F55D855D688035E53875F0B1
:104582000884FF7E008F5DE53875F00884ADF07C0D
:10459200008D607565087533037534B6E55DC394A7
:1045A2001F50051238E5800690045BE0F55D855DDD
:1045B20068229000F8E0F562756511753304753470
:1045C20000AE25AF26E56275F00FA4FDACF0EDD389
:1045D2009FEC9E4021E5628E048F05FF120085ED5F
:1045E20075F010A4FFAEF0E53875F01184FD7C0083
:1045F200ED2FF563800EE53875F01184FF7E00EF34
:1046020024F0F56385635DE53875F01184AFF07EC3
:10461200008F601238E5855D64AE25AF269000F804
:10462200E075F00FA4FDACF0EDD39FEC9E40287531
:10463200330475341085635D1238E585645E855DEB
:104642005FAE25AF26E5628E048F05FF12534A8DB9
:104652006085626112395F855D67756864229000CA
:10466200F8E0F562756511753304753400AE25AF57
:1046720026E56275F00FA4FDACF0EDD39FEC9E40F1
:1046820021E5628E048F05FF120085ED75F010A4FE
:10469200FFAEF0E53A75F01184FD7C00ED2FF56375
:1046A200800EE53A75F01184FF7E00EF24F0F56389
:1046B20085635DE53A75F01184AFF07E008F60127C
:1046C20038E5855D64AE25AF269000F8E075F00F01
:1046D200A4FDACF0EDD39FEC9E40287533047534F5
:1046E2001085635D1238E585645E855D5FAE25AF3A
:1046F20026E5628E048F05FF12534A8D6085626142
:1047020012395F855D677568649000F3E0B40479DF
:10471200900058E0FE9000C2E0D39E4037E5387525
:10472200F00884FF7E008F5DE53875F00884ADF0F7
:104732007C008D60756508753303753496E55DC33D
:10474200941F50051238E5800690043BE0F55D8524
:104752005D688035E53875F00884FF7E008F5DE581
:104762003875F00884ADF07C008D6075650875338E
:10477200037534B6E55DC3941F50051238E5800613
:1047820090045BE0F55D855D682290008CE0B401E9
:104792003BE54075F00584FF7E008F5DE54075F0D6
:1047A2000584ADF07C008D60756505753305753443
:1047B20018E55DC3941750051238E580069005B5DB
:1047C200E0F55DE568255DC39464F56890008DE0D1
:1047D200B4013BE54175F00584FF7E008F5DE54144
:1047E20075F00584ADF07C008D6075650575330547
:1047F200753460E55DC3941750051238E580069064
:1048020005FDE0F55DE568255DC39464F568E5673F
:104812002568F55A900094E0B402109007CAE0258A
:104822005AFE9000E8E0F4042EF55A9000EBE0D333
:1048320094014040E544C394E7501D74E7C3954496
:10484200FE9007CCE08E00F5F0E884FF7E008F5DDD
:10485200E55A255DF55A801CE544C394E7FE9007AE
:10486200CCE08E00F5F0E884FF7E008F5DE55AC350
:10487200955DF55AA2084006E5672464F55AE55AA3
:10488200D394644009E55AC39464F55A8003755A77
:10489200009000C4E0C3955A50069000C4E0F55A57
:1048A20022D2009000DAE0A825B800049526503BF9
:1048B2009000DAE0A825B8000495265003755A0F37
:1048C2009000DAE004A825B8000495265003755A32
:1048D2000A9000DAE02402A825B8000495265005C3
:1048E200755A05C200740990005BF07E017F00904A
:1048F20000CAE012532F9000D9E08E048F05FF12F8
:104902000085E538BC000CD39D4008C200740A90B3
:10491200005BF09000CBE0C39540500D9000DDE0CD
:10492200A825B80006952640028008C200740B90A4
:10493200005BF0A2004003755A05900094E0B403B6
:1049420006A201B3B34002802B900080E0C394051D
:10495200A825B800049526500C9000B5E0F55A74CD
:104962000C90005BF0900080E0A825B8000495262A
:104972005002C200855A45900086E0255AFE9000FA
:1049820058E075F01E84FC7F00EE2CF55A22900050
:1049920058E075F00584FF7E008F5D900058E07549
:1049A200F00584ADF07C008D607565057533037587
:1049B20034D69000D7E01475F00584FF7E00E55DE3
:1049C200BE00039F50051238E5800BE55D90045C44
:1049D20012536BE0F55DE55D9007CDF09007CDE0F9
:1049E200FE9000C6E0C39E50089000C6E09007CD3E
:1049F200F022E54075F00584FF7E00900586125393
:104A020056E0F56CE56CD394644010E56CC3946495
:104A120075F00F84FF7E008F6C8003756C00900030
:104A2200A9E0256CF56C229007C0E0FEA3E0FF74BC
:104A320004125321E53812532F740F8E048F05FF91
:104A42001200859007BEECF0A3EDF090009CE0B45C
:104A52000262E543C3944175F00584FF7E008F5DD9
:104A6200E54375F00584ADF07C008D6075650575D4
:104A72003306753414E55DC3941750051238E5808A
:104A8200069006ADE0F55D9007BEE0FEA3E0FF7480
:104A92000A8E048F05FF120085E55D8C068D0712D4
:104AA200532F740A8E048F05FF1200859007BEEC07
:104AB200F0A3EDF09007BEE0FEA3E0FF9007C4E094
:104AC200FCA3E0FDEDD39FEC9E400F9007C4E0F8FD
:104AD200A3E09007BEC8F0A3C8F0229000A3E0B400
:104AE20001038526509000A3E0B402129000D9E0A1
:104AF2008538F0A4FFAEF074081253218F50900055
:104B0200A3E0B40303853A509000A3E0B404038504
:104B120040509000A3E0B40507E541C39414F5505A
:104B22009000A3E0B406038542509000A3E0B407CE
:104B3200038543509000A3E0B408038544509000DD
:104B4200A3E0B40903853F509000A4E0FE9000A5C5
:104B5200E0D39E404B9000A3E0B404189000A5E07F
:104B6200C395505002D2049000A4E0D39550400265
:104B7200C204802A9000A4E0C3955050099000A579
:104B8200E0D3955050028002D2049000A4E0D39565
:104B92005050099000A5E0C395505002C204802AEB
:104BA2009000A4E0D3955040099000A5E0C3955031
:104BB20040028002C2049000A4E0C39550400990D4
:104BC20000A5E0D395504002D204229000A6E0B4A2
:104BD20001038526509000A6E0B402129000D9E0AD
:104BE2008538F0A4FFAEF074081253218F50900064
:104BF200A6E0B40303853A509000A6E0B40403850E
:104C020040509000A6E0B40507E541C39414F55066
:104C12009000A6E0B406038542509000A6E0B407D7
:104C2200038543509000A6E0B408038544509000E9
:104C3200A6E0B40903853F509000A7E0FE9000A8CB
:104C4200E0D39E40409000A7E0C3955050099000E9
:104C5200A8E0D3955050028002D2069000A7E0D37C
:104C6200955050099000A8E0C395505002C206909A
:104C720000A6E0B401099000E5E0D3953A50028025
:104C820002C206802A9000A7E0D395504009900006
:104C9200A8E0C3955040028002C2069000A7E0C37C
:104CA200955040099000A8E0D395504002D20622C8
:104CB200AE58AF5974F5D39F74019E4008785812CC
:104CC2005396024DAD755901755800AE25AF26E5D4
:104CD2006CBE000DD39F40099000BBE0D3956D40A0
:104CE20002801B756D00E56CC39526F5509000BEE1
:104CF200E0D3956B4006E56B2550F56B8002056DA0
:104D0200900097E0D3953A401CE538D39539401589
:104D1200AE25AF26E56CBE00039F50099000BCE0B3
:104D2200D3956E400280579007CEE0A825B80004C4
:104D3200952650037570009007CEE0A825B8000BA9
:104D4200D395264006E5269007CEF0E570702AE559
:104D520026C3956CF550E550D39405400375500574
:104D62009000BDE0C3956B5007E550C3956B4002C0
:104D72008007E56BC39550F56B756E008002056E7A
:104D8200E5707016900097E0C3953A500DE56C24DB
:104D920005A825B8000695264002800F9000AAE0DB
:104DA200F56B75700174789007CEF022AE58AF594A
:104DB20074E9D39F74039E40087858125396024FA9
:104DC2005B755901755800756B32A222402A756BCA
:104DD200199000AAE075F002A4FFAEF0E56DBE00E6
:104DE20006D39F4002D222056D7570037478900736
:104DF200CEF0756F00024F4AAE25AF26E56C6F4EBE
:104E02007003024F4AE56CBE000DD39F400990002B
:104E1200BBE0D3956D40028017756D00A208B3B355
:104E22005007E570C3940340028003756B19800D2F
:104E3200E56CC39526F550E56D2550F56D9000970C
:104E4200E0D3953A400E9007CEE0A825B80007D3EC
:104E520095264002800C056F9000AAE0B56F03759D
:104E62007000E570B4030DE56C2402A825B80006B5
:104E720095264002800A056FE56FB43C0375700207
:104E8200E570B402299007CEE0A825B8000ED395AC
:104E9200264009E5269007CEF0756F00900097E056
:104EA200C3953A5009756F0074789007CEF0E5709B
:104EB200705A900097E0D3953A401CE538D3953963
:104EC2004015AE25AF26E56CBE00039F5009900049
:104ED200BCE0D3956E40028008756E00756B4B8006
:104EE20028E526C3956CF550E550D394054003752B
:104EF2005005900097E0D3953A4008E56E2550F5AD
:104F02006E8006E56E2406F56E756F00E57070160C
:104F1200900097E0C3953A500DE56C2405A825B89A
:104F22000006952640028003757001E570B40118F1
:104F3200756B19056F9000AAE0B56F067570027562
:104F42006F0074789007CEF0E56B75F00AA4FFAE9F
:0A4F5200F09007C8EEF0A3EFF02284
:09536B002582F58250020583221F
:0F53120025E050020583258250020583F5822293
:10006400EF2F500205832582F582E5833E2EF5832A
:010074002269
:10538600CFC39FFF50011E22C3EF9DFFEE9CFE225E
:09537400E493F608740193F6229B
:085396000806B6000218062209
:0D533D00A3E004F07006125361E004F022BA
:0E003900A3E014F0B4FF06125361E014F022AD
:0E532100048007C3CE13CECF13CFD5E0F62203
:10523100BC000FBE0008ED8FF084FFADF022E4FE4C
:10524100FF22BE000DEF60FE54F0606F20E7030205
:1052510052E7EAC0E0EBC0E078017A0075F001EEB8
:1052610020E710EF25E0FFEE33FE0AC5F023C5F07D
:1052710030E7F0EA5407F9096A7A007B0060010817
:10528100C3EC9E40167004ED9F4010ED9FFDEC9E17
:10529100FCE5F0CA4ACA03F5F08005E5F003F5F034
:1052A100C3EE13FEEF13FFD9D77908CACBCAD8D002
:1052B100EAFEEBFFD0E0FBD0E0FA22EC8FF084FCB9
:1052C100ED54F045F0C48FF084FEEDC454F045F088
:1052D100C48FF084FDEEC4FE54F02DFFEE540F3C5C
:1052E100FEADF07C0022790078008FF0EC7E082082
:1052F100E70DC3CD33CD33C933C9C833C8DEF0841C
:1053010049F9E5F08FF0BE00E6FD7C00E9FFE8FE1B
:015311002279
:0E532F00F88FF0A4FFE5F0CE88F0A42EFE2249
:10000300EF8DF0A4F9A8F0EF8CF0A428F8EE8DF0B2
:06001300A428FEE9FF2213
:10007500600D782B02007F007830D8FED5E0F8229D
:10008500EEC0E07E00125231EFFDEEFCD0E0FE2224
:0C534A00EEC0E07E00125231D0E0FE22E6
:03001B0002001EC2
:03009B0002004917
:0300000002537D2B
:09537D0075817175D0000206A0D3
:10535600E5822FF582E5833EF583220582D582021A
:055366001583158222F1
:10001E00C0E0C0F0C083C082C0D075D00012066DA3
:0B002E00D0D0D082D083D0F0D0E032E0
:10004900C0E0C0F0C083C082C0D075D00012067075
:0B005900D0D0D082D083D0F0D0E032B5
:00000001FF
